:020000040000FA
:0400000072303A28F8
:08000800A000030EA100831209
:100010008B1C32288B1031181428B11C3228643004
:10002000010203183128182800001628172818285C
:1000300019281A281B281C281D281E281F283110A3
:10004000B114A810031005190314AA0DA90DA80DC9
:10005000B00B322831152A08AF002908AE00280855
:10006000AD00B11081010B11210E8300A00E200EF6
:02007000090085
:0C007400203084008001840A6030040207
:10008000031C3C281230B00056218316FF23900039
:10009000831283160C308505870183128501870141
:1000A000073099000030831691009F008312C830FA
:1000B00083168100831231309000003083168C004B
:1000C000831210308B00872181018E018F010B116B
:1000D0008B100B108C018B177C20311992203A2148
:1000E000B30B7A28031085190314B90DF0303902C7
:1000F0000319E32088216C286400311808000B1DC7
:1001000008000B11B11031141230B000051D8D28FC
:10011000321483160113831208003210831601175C
:100120008312080031110130B7008B1320303707DC
:1001300083169B001C141A088312A400A500C0306B
:10014000A5061030370783169B001C141A0883126B
:10015000A3000030370783169B001C141A08831273
:10016000A2008B17321CBA2822090339A200A30966
:10017000A409A50922082D02031DDD2823082E024B
:10018000031DDD2824082F02031DCF28013037026C
:10019000031DCF283D18CF283D143E146E2125089D
:1001A0002F02031DDD2801303702031DDC283D1C12
:1001B000DC283D103E147121DD28B70A02303702D9
:1001C0000318080095280130B600B300B400B5004C
:1001D000B70085018701B1137D217C20B30B08296D
:1001E000031085190314B90DF030390203192F29B2
:1001F000B41F8501B41F8701B40B0829B50B08296A
:100200000230B50001303702031974219630B40072
:10021000311DED283111321C12292D090339AD0091
:10022000AE09AF092F1CB1132F1CED28B11BED280F
:100230002E18ED28B1178B1320303707BB002F087D
:10024000BA00432110303707BB002E08BA00432103
:1002500000303707BB002D08BA0043218B178421DB
:1002600085018701B70AB60102303702031CED2869
:10027000872108003E1C08003E101030BB003D08DE
:10028000BA00432108008B133A0883161C159A0004
:100290003B089B0055309D00AA309D009C146400D3
:1002A0009C184F291C1183128B17080083161030DD
:1002B0009B001C141A088312BD00FF30D4000230CA
:1002C000D5000C30D600BA30D7003730D800DA303D
:1002D000D9006F30DA00B830DB0008000130BD0013
:1002E0000800850187010800380933398500B80006
:1002F0003F093F398700BF00080011308500B80072
:1003000013308700BF000800B801BF0108000800D3
:1003100001303D05031908005C180516DC18851628
:100320005C190514DC1985145C1A8714DC1A07158E
:100330005C1B0714DC1B87165D180716DD18871574
:10034000E6300E02031CAE29051685160514851429
:100350008714071507148716071687158F080319C2
:1003600008008F01850187015408DE003B22D4007C
:100370005508DE003B22D5005608DE00541C3B2207
:10038000D6005708DE00D41C3B22D7005808DE00F8
:10039000541D3B22D8005908DE00D41D3B22D90051
:1003A0005A08DE00541E3B22DA005B08DE00D41E31
:1003B0003B22DB00CA0BE4295408CA00D4185C14A1
:1003C000D41E5C10D41D5C10CB0BEE295508CB005D
:1003D000D51ADC14551DDC10551FDC10CC0BF82988
:1003E0005608CC00561A5C15561F5C11D61D5C11C0
:1003F000CD0B022A5708CD00571ADC15D71FDC1188
:10040000D71DDC11CE0B0C2A5808CE00D81B5C1669
:10041000D81F5C12D81C5C12CF0B162A5908CF00CB
:10042000591ADC16591EDC12D91FDC12D00B202AF7
:100430005A08D000DA195C17DA1D5C135A1E5C13D7
:10044000D10B2A2A5B08D1005B1ADC175B1EDC1378
:10045000DB1FDC13D20B322A5608D200D51B5D14E9
:10046000D71F5D10D30B3A2A5708D300D61BDD14D3
:10047000D81FDD100800C001DE080319DE035E1876
:100480004014DE1A40144008C0015E1C4014DE1EF9
:0A0490004014C005C00C5E0C08000B
:084000000F0003000600070099
:02400E00CC01E3
:10420000010003000300030003000200020002009B
:1042100002000000000000000000FF00FF00FF009F
:10422000000000000000000000000000000000008E
:104230000000C000C000C000C000FF00FF00FF0081
:104240000100C300F300CF00FF00C300F300CF0064
:10425000FF00C300F300CF00FF00FF00FF00FF00DE
:10426000FF00FF00FF00FF00FF00FF00FF00FF0056
:10427000FF00FF00FF00FF00FF00FF00FF00FF0046
:10428000FF00FF00FF00FF00FF00FF00FF00FF0036
:10429000FF00FF00FF00FF00FF00FF00FF00FF0026
:1042A000FF00FF00FF00FF00FF00FF00FF00FF0016
:1042B000FF00FF00FF00FF00FF00FF00FF00FF0006
:1042C000FF00FF00FF00FF00FF00FF00FF00FF00F6
:1042D000FF00FF00FF00FF00FF00FF00FF00FF00E6
:1042E000FF00FF00FF00FF00FF00FF00FF00FF00D6
:1042F000FF00FF00FF00FF00FF00FF00FF00AA001B
:00000001FF
